:020000040001F9
:10C000003834002071C201008BC201008DC20100D2
:10C010000000000000000000000000000000000020
:10C020000000000000000000000000008FC20100BE
:10C03000000000000000000091C2010093C2010056
:10C0400095C2010095C2010095C2010095C2010090
:10C0500095C201000000000029D7010095C201002F
:10C0600095C2010095C2010095C2010095C2010070
:10C0700095C2010095C2010095C2010095C2010060
:10C0800095C20100DBCF010095C2010095C20100FD
:10C09000F1CF010095C2010093DA010095C20100C1
:10C0A00095C2010095C201000000000000000000E0
:10C0B0000000000000000000000000000000000080
:10C0C00000F002F800F03EF80CA030C80838241840
:10C0D0002D18A246671EAB4654465D46AC4201D1C0
:10C0E00000F030F87E460F3E0FCCB64601263342B4
:10C0F00000D0FB1AA246AB4633431847003300007A
:10C1000020330000103A02D378C878C1FAD8520719
:10C1100001D330C830C101D504680C6070470000FD
:10C120000023002400250026103A01D378C1FBD853
:10C13000520700D330C100D50B6070471FB51FBD3B
:10C1400010B510BD03F00AF91146FFF7F7FF00F034
:10C15000C8F803F022F903B4FFF7F2FF03BC03F0C1
:10C1600029F90000026882F3088843681847000034
:10C17000401E00BF00BF00BF00BF00BF00BF00BF28
:10C1800000BF00BF00BF00BF00BFF1D1704700007B
:10C1900070B505460C46164602E00FCC0FC5103EA2
:10C1A000102EFAD2082E02D303CC03C5083E042E6B
:10C1B00007D301CC01C5361F03E021782970641C28
:10C1C0006D1C761EF9D270BD234922480860704765
:10C1D00010B500F01DF8002805D021491F4848601F
:10C1E000C813204988612048018CC9B201290ED1A9
:10C1F000818C09070BD1018D0906090F042906D18D
:10C20000808D0006000F02D118490120886010BD02
:10C210001548018CC9B2012917D1818C090714D1A5
:10C22000018D09060A0F03D1828D1206120F0ED05E
:10C23000090F012903D1828D1206120F07D003299D
:10C2400003D1808D0006000F01D00020704701202F
:10C25000704700000024F40000200020DFFF07C02A
:10C2600000050040006C0040C00F00F000060040D8
:10C2700003210C4802680A4302600B4802680A4323
:10C2800002600A4880470A480047FEE7FEE7FEE7EB
:10C29000FEE7FEE7FEE7000006480749074A084BAD
:10C2A000704700002405004054050040D1C1010042
:10C2B000C1C001003828002038340020382C00206C
:10C2C000382C002001207F49C003886000F08BF8E3
:10C2D0000A4601467C48FFF7F5FF10B501F04EFD18
:10C2E00010BD08B5794903200860091F0860774A26
:10C2F000183A10600860764807214069890388422F
:10C3000013D10120000700690121890288420FD161
:10C3100070480090704B05220321002000F08EFE33
:10C3200000280AD06DA29D2105E06CA2EC2101E05D
:10C330006AA2ED210020FFF7C5FF674901201439EB
:10C3400001F04CFA002802D064A29221F3E75F4981
:10C35000032000040831086000F05BF8624A1421F1
:10C36000082001F0E7F8002802D05CA2DF21E2E714
:10C37000544D28695D4C800CC007C00F04D0204686
:10C3800000F00BFA00280CD101200004A86000F096
:10C3900084FA002802D051A2FE21CCE7102000F040
:10C3A0002AF8204600F0F9F900280ED0102000F0FD
:10C3B00022F80F2000F01FF80A2000F01CF80F20D0
:10C3C00000F019F8204600F094FA102000F013F85D
:10C3D0000F2000F010F80A2000F00DF80F2000F0F8
:10C3E0000AF800F000F8BFF34F8F42494048C86098
:10C3F000BFF34F8FFEE7012181403248C160704793
:10C400001CB5019100903C4A0821684601F0A6F84D
:10C410001CBD00B5394B85B00FCB03936B4607C3EA
:10C42000684618DF002802D02CA2C42125E007208E
:10C43000800313DF002802D028A2C7211DE02A496B
:10C440002F4B502250390B2001F0F6FA002802D071
:10C4500022A2CB2111E0002069460490087404A8B0
:10C4600060DF002802D01DA2D32106E0254801F09C
:10C4700008FB002803D019A2D721FFF723FF05B03E
:10C4800000BD10B50246082905D0FF211EA21B31B0
:10C490000020FFF717FF11685068884710BD10B5DE
:10C4A0000021254A084601F059F810BD10B50029B1
:10C4B00004D022A299210020FFF704FF01F07EFAA8
:10C4C00010BD000000050050EFBEADDE400700507B
:10C4D0000010001001C40100FC2000202E2E5C6D15
:10C4E00061696E2E630000008C2300200060010053
:10C4F0000400FA0500ED00E083C40100DCF3010054
:10C500009FC40100DBC201002E2E5C2E2E5C2E2E5D
:10C510005C2E2E5C2E2E5C496E636C7564655C61CE
:10C5200070705F636F6D6D6F6E5C6170705F74696A
:10C530006D65722E68000000ADC401002E2E5C2EC9
:10C540002E5C2E2E5C2E2E5C2E2E5C496E636C753E
:10C5500064655C73645F636F6D6D6F6E5C736F6653
:10C56000746465766963655F68616E646C65722E7C
:10C5700068000000F8B5784C1F46606815460E4606
:10C58000042809D1022E0ED1002D0CD12269002AD7
:10C5900009D01946284690476068012803D1042E27
:10C5A00001D1002D06D0280003D06CA25321FFF743
:10C5B00089FEF8BD6269002AFBD00220606039461E
:10C5C00028469047F8BD70B5634C01206060002597
:10C5D00025706949658067480860214618316648BA
:10C5E00001F0FCFD002801D0656070BD0B205A49A8
:10C5F000400318314860002070BD574908617047FA
:10C6000055494861704770B504460320082540032A
:10C61000844201D90C2070BDA00701D0062070BD56
:10C620004D4E706801280DD130462146183001F07A
:10C6300021FE0500F3D1B460F0603A4601201146B6
:10C6400000F0E4F8284670BD70B5002804D0816879
:10C650008A0703D0102070BD0E2070BD3E4C62686A
:10C66000022A05D0032A03D0042A03D0082070BD73
:10C67000042262604068E3688500A268581990420D
:10C6800001D90C2070BD34482A46183001F0C2FD93
:10C690000028F7D1E1684919E160A2689142F1D020
:10C6A000092070BD70B52C494A68022A02D0032ABD
:10C6B00005D101E003224A60CA68002A01D008209F
:10C6C00070BD2D4C0022403C08E0836895005D5908
:10C6D0000B789E005B1CA5510B70521C4368934263
:10C6E000F3D8002070BD10B51B4C6068042819D128
:10C6F00005206060A168E068884213D10B20002209
:10C70000400301F037F91C496080403922780988DC
:10C71000002A03D0884201D00B2010BD06206060A3
:10C72000002010BD082010BD0EB50B494868062832
:10C7300001D008200EBD002000904A886B469A80E8
:10C740008A680292019900F061F800200EBD10B5D0
:10C75000042000F05BF810BD042000202E2E5C6445
:10C7600066755F73696E676C655F62616E6B2E6381
:10C770000000000075C501001C25002010B57C4894
:10C780000368012B02D1022900D10160100003D0FF
:10C7900078A23421FFF796FD10BD38B50B25002493
:10C7A0006D03A84215D1684600F0FEF800980168B4
:10C7B00001290ED18188002908D0C16800222846AD
:10C7C00001F0D8F800998988814201D1012400E064
:10C7D0000024204638BD10B5044665481021001DD0
:10C7E00001F0B2FC002803D062A28521FFF76AFDA8
:10C7F0005F48002310222146001D01F0D1FB0028D4
:10C8000003D05CA28B21FFF75DFD10BD17B581B091
:10C81000684600F0C9F801995A48554C002913D0D0
:10C8200003291CD0FE22012923D002292CD004295F
:10C8300009D101F0DEFE002803D04EA2BE21FFF791
:10C8400041FD042020601FBD69460989818003994C
:10C85000C1600121FF2282600160216010E001F0CF
:10C86000C8FE002803D043A2A421FFF72BFD03201C
:10C87000E8E7002181800260C160009989688160D9
:10C880004048FFF7A8FF1FBD00990B6803608B8825
:10C890008380C9688260C160F2E73EB53A48009083
:10C8A000102001900120029001F0CEFA00281FD143
:10C8B0002F496846091D01F0F0FA002818D1FFF74A
:10C8C00082FE002814D101F086FF0546284C40DF87
:10C8D000002803D02DA24621FFF7F4FC00F0B4FE9F
:10C8E0002068022803D0032801D00428EFD128466D
:10C8F0003EBD70B511DF002804D0FF211DA20A3112
:10C90000FFF7E0FC254900200B68244C012180340E
:10C910000A4682401A4204D0C506ED0E0A46AA40D5
:10C920002260401CC0B22028F2D30B2464032046AE
:10C9300013DF002804D0FF210EA21431FFF7C2FC40
:10C94000204600F02DF870BD1FB5094904460023AC
:10C950001022091D684601F0A9FB00982060684676
:10C960008088A0800398E0600298A0601FBD00004E
:10C97000242000202E2E5C626F6F746C6F616465E2
:10C98000722E6300282500207DC701002E2E5C62D8
:10C990006F6F746C6F616465722E630000E100E07C
:10C9A00010B5FFF7DFFB10BD0149016070470000C3
:10C9B00000FC010030B585B0002822D00388FB4C74
:10C9C000A34220D0FA4B1B78002B1CD0F84B10252B
:10C9D0005B1C1D705970002401259A700322694662
:10C9E0000A820094019402940394C2890A808D7093
:10C9F0008C8004A90291039300886946A6DF05B0E4
:10CA000030BD0E20FBE70820F9E7F0B589B00446F9
:10CA10000227684607700D468783608A08AB07AA1D
:10CA20000021A5DF0026002804D0616A00291AD061
:10CA3000884718E06846008CC007C00F13D06846CE
:10CA4000868020886946A8DF002812D1A97E284662
:10CA500001221B300B0002F0B4FC093F0E1E202205
:10CA600024263D283F00FF20FE306946888020882C
:10CA7000A8DF09B0F0BD0496298B022902D26846CE
:10CA8000067502E069460A750690226A04A92046E6
:10CA900090470020EDE70492F7E70497F5E70320BD
:10CAA00014E0042012E0052010E0298B032905D2B0
:10CAB000032208212046FFF77DFFDAE7417802785C
:10CAC000080210436946888202D006200490DCE701
:10CAD0000720FBE70920F9E70322EBE730B585B033
:10CAE0000D46040032D0002D30D0286800282DD00B
:10CAF0000020C043AF4B20800FCB049301AB07C392
:10CB0000AD486946088001A8811E63DF00281CD15A
:10CB1000A21C69460120A0DF002816D16846807853
:10CB20002071204600F0C0F800280ED1204600F009
:10CB3000FBF8002809D1286820626868002800D026
:10CB400060629B4901200870002058E70E2056E7DC
:10CB50003EB5002820D000291ED0026A002A1BD032
:10CB60000A88102A19D0112A28D0502A17D0512A01
:10CB700012D104468879891D02280DD14888E2899E
:10CB8000904209D12046891CFFF73FFF002803D0BF
:10CB9000616A002900D088473EBD898810E0CA88B4
:10CBA000C3889A42F8D1082200928A7F6B461A7194
:10CBB00020310291026A694690473EBD0021C94377
:10CBC00001803EBDF0B585B00A4605002DD028880D
:10CBD000764988422BD076480078002827D0744CBC
:10CBE0001020641C2070072060700127A7700321AB
:10CBF000684601820026E11C104600F04CF8014610
:10CC00006846008A091868460182009601960296D5
:10CC10000396E98901808770868004A803940290B6
:10CC200028886946A6DF05B0F0BD0E20FBE7082086
:10CC3000F9E7F0B585B00A46050028D028885B4999
:10CC4000884226D05A480078002822D0584C11201B
:10CC5000641C20700127684607820026611C10466C
:10CC600000F019F801466846008A091868460182F2
:10CC70000096019602960396E98901808770868066
:10CC800004A80394029028886946A6DFCBE70E200B
:10CC9000C9E70820C7E70870020A4A70020C8A70C8
:10CCA000000EC8700420704730B58FB005461C21B7
:10CCB000684602F090FA69460878042108436946FC
:10CCC0000870002401940394049405940694287930
:10CCD00008A9887038486946801C0884601C0007D1
:10CCE0000794000F0C77103048778A7FF9200240B4
:10CCF000F720921C0240EF200240012002438A7775
:10CD0000142109A802F067FA08A8099007A80A9058
:10CD100069468C851420CC8508860D946888AB1DE7
:10CD200009AAA2DF0FB030BD30B58FB005461C2177
:10CD3000684602F050FA6946087808210843102234
:10CD400010436946087000240194039404940594E8
:10CD50000694287908A9887017486946401C0884F9
:10CD6000601C00070794000F0C7710304877887F0D
:10CD7000F9210840F721801C084010430121084395
:10CD800069468877142109A802F025FA08A80990B5
:10CD900007A80A9069468C851720CC8508860D94D3
:10CDA0002B4668880E3309AAA2DFBBE7FFFF00000D
:10CDB00030200020ECF30100301500008307FF2233
:10CDC000DB0E9A408907090E994000280BDA00070C
:10CDD000000F08388308FF489B001818C369934365
:10CDE0000B43C36170478308FB489B001B181868FE
:10CDF000904308431860704770B50124F7496004F8
:10CE00000860F74940108860F54940398860F54D61
:10CE10006C602F20FFF7ACF9AC60F34D00242F209D
:10CE20006C61FFF7A5F92C7170BDF0B5EE4F2821AC
:10CE3000BC6841430D1939694A1C09D028224A436C
:10CE40001619AB68B268934204D8D21AB26069620C
:10CE50003861F0BD0A4602E00A46796A9B1B4E1C07
:10CE60000BD028264E433719BE689E42F4D328269D
:10CE70004E433619B768FF1AB760AB606962282164
:10CE80004A4311194862F0BDF8B5D74C2569681CB2
:10CE900036D0D648002640686169401A07023F0A2A
:10CEA0001AE028204543A0682A189068B84215D88F
:10CEB000A3693F1A8619556A002B0AD0116AD069F6
:10CEC0009847002808D0FF21C9A26431FFF7FAF97A
:10CED00002E0D169106A8847681CE2D1A178E07845
:10CEE000814206D1401CC0B2E070022801D100206E
:10CEF000E070BD490006800D1C310E5000F0F2F9C3
:10CF0000F8BDF8B50446B84801690091467856E086
:10CF1000B548F100C2688D184BE0601C07D0B24ADA
:10CF2000282192686143204689184C6A20E02878BD
:10CF3000182141436A68401CC0B252182870A97871
:10CF4000884201D100202870A74B506828219B6897
:10CF50004143C9181368012B2DD10B7E002B2AD118
:10CF60009368CB60D3680B6113694B6152690A62A5
:10CF70009D4ACF685369BC46FA1A1202A84F120A9A
:10CF8000BA4202D20B69D21809E062469A1A12021A
:10CF90000B69120A934201D99A1A00E000228A60B2
:10CFA0000022CA600A6101220A76921E4A62FFF7D5
:10CFB0003CFF601CB1D1287869788842ADD13046F9
:10CFC000761EF6B20028A3D18748016900988142F5
:10CFD00001D00120F8BD0020F8BD92490020086072
:10CFE00048608860C8608F494039086048604BE7F6
:10CFF000F0B5002087B0C04302907B4846690569C0
:10D00000684600F074F9074600F08EF90446002FD8
:10D0100008D002AA3146009800F0CEF90298FFF736
:10D0200070FF06E00298FFF76CFF002801D1002C8A
:10D0300002D0284600F0E9F907B0F0BDFFB5980727
:10D04000002481B01E4615460F4600280BD1002E45
:10D0500009D0FFF7D1FE64490A9888610F70324603
:10D0600000208E6008E0072005B0F0BD2823434370
:10D07000D4509B181C76401CB842F7DB282047434D
:10D08000BB19032048700F461846CB60194618306C
:10D09000002218232E465E43D3005B181C705C7080
:10D0A0009D7058603018521C032AF5DB0020C043E5
:10D0B0003861BC70FC7001245B48240504600321C6
:10D0C0001420FFF77BFE454880380460474C0198E8
:10D0D000A06003211120FFF771FE606878610020D5
:10D0E000C2E770B5404CA568002D06D0002A06D0D6
:10D0F000002804D00023247809E0082070BD072010
:10D1000070BD28265E43AE59002E04D05B1CA3429E
:10D11000F7DB042070BD282401265C432E516419DE
:10D12000E26161600360002070BD2A494868C00563
:10D13000C00D17D0103807D50207120F083A920811
:10D1400092005118C96904E08108234A89008918AE
:10D1500009688007C00EC1400806800F012803D06F
:10D16000032803D002207047002070470120704739
:10D17000FEB504461C48174682680D46002A0CD0AE
:10D1800001788C4201D2052D01D20720FEBD214637
:10D19000282359435358012B01D00820FEBD88187D
:10D1A0004068012848D00026FFF7BFFFC0000E49A5
:10D1B0000190C9684018694600F06DF900283DD01B
:10D1C000012112C009494968E2C007490198C968AC
:10D1D00041182BE000ED00E000E400E080E100E019
:10D1E000401301400010014038200020001501408C
:10D1F0002E2E5C2E2E5C2E2E5C2E2E5C2E2E5C5344
:10D200006F757263655C6170705F636F6D6D6F6E7B
:10D210005C6170705F74696D65722E630000000060
:10D22000FFFF7F004011014080E200E0009848705D
:10D2300000F058F80020FEBD2E46B5E70420FEBDE4
:10D24000F8B5B64D0446A868002809D029788C4264
:10D2500001D30720F8BD282161434058012801D09F
:10D260000820F8BDFFF761FFC600E868694630187E
:10D2700000F011F9002809D0022112C0E868311825
:10D280000098487000F02EF80020F8BD0420F8BD8A
:10D2900038B5A24CA068002815D0FFF746FFC5009E
:10D2A000E0686946281800F0F6F800280DD0032140
:10D2B0000160091F4160E06829180098487000F07B
:10D2C00011F8002038BD082038BD042038BD94492D
:10D2D0004968016000207047401A0002000A10608F
:10D2E0000020704701208F4900050860704710B585
:10D2F0008A4900238A78CC78A24212D0521CD2B23A
:10D300008A70022A00D18B708A78844B92001C3379
:10D310009A580260486910180002000A486101200A
:10D3200010BD0360002010BDF8B57C480169009174
:10D33000457833E07948E900C0680E1834782AE06F
:10D34000182060437168641C0818B178E4B2A142E7
:10D3500000D100240168022902D003291BD113E067
:10D360006E4A40682821926841438F18397E00290F
:10D3700011D000F0A2F8002038760CE0282778437E
:10D38000C0180276406A03E0644900228B6808698D
:10D39000471CF3D108617078A042D1D128466D1E98
:10D3A000EDB20028C6D15D4801690098814201D0E4
:10D3B0000120F8BD0020F8BDF7B5584C0025A7683E
:10D3C00023691EE028215943C9198E68864202D973
:10D3D000301A886017E0801B751900268E600E7663
:10D3E0004E699C464B6AB646002E0AD0019E7619BD
:10D3F0003602360ACE6076460E6116684E62614687
:10D400001160591CDED12361FEBDF8B543480169A6
:10D410004A1C3DD028225143826889188E684049B1
:10D420004C6847690079E11B0D022D0AED1C0028AC
:10D4300015D101203C4A000450603B4A403A5060FC
:10D440003849400080310860384908603849012077
:10D4500008602F20FEF78CFE304901200871B5428C
:10D4600000D23546E81900022D49000A4031086013
:10D470002B494968001B091B0902090A0002000A1E
:10D48000C91C814203D90120264940040860F8BD27
:10D49000FFF7B2FCF8BD42788378521C934200D16A
:10D4A00000220378934201D1002070470A6041684E
:10D4B0004078182250430818704770B5174E3569E8
:10D4C000B26829460C4606E0844207D02546282348
:10D4D0005C43A3185C6A631CF6D170BD002BFCD0C2
:10D4E000A54208D1282041438818406A3061401C79
:10D4F00001D1FFF781FCB16828204443601828233C
:10D5000082685D43406A6B185862431CE5D028234B
:10D510005843401881688918816070BD3820002008
:10D520000015014000E200E04013014000E100E08E
:10D530000010014030B5CB0008339DB293070024A2
:10D54000002B01D0072030BD564B9A605219DA608B
:10D550005C701C7058809980002030BDF7B5514C2C
:10D5600082B060880F4681426CD8002069460870FE
:10D570004E494D4E4868C005C00D16D0103807D52D
:10D580000207120F083A920892005118C96904E084
:10D590008108474A8900891809688007C00EC14080
:10D5A0000806850F012D01D10AE0042568462EDF0B
:10D5B00002280BD0002803D03EA25921FEF782FE9C
:10D5C0006078A188884203D2401C02E072B6F7E777
:10D5D00000202278C0B2904207D0667860788842F6
:10D5E00001DA401C00E000206070012D0BD062B613
:10D5F000684600782FDF022805D0002803D02DA22E
:10D600006121FEF75FFE2848864219D0A068F50028
:10D6100004994151029900290CD0002F0AD060884A
:10D620003A464643E068301801F076FDA0682818B5
:10D63000878002E0002128188180002005B0F0BD1D
:10D640000420FBE70920F9E70EB504E0684681886D
:10D65000029A0098904702AA01A9684600F003F8D0
:10D660000028F3D00EBD70B50E4B05245D781E78F2
:10D67000B54215D01D781C789E88B44201DA641C2E
:10D6800000E000241C705C88DE686C43A419046010
:10D690009B68E800C418A4880C8018580024106007
:10D6A000204670BD5C200020FFFF000000ED00E080
:10D6B00000E400E02E2E5C2E2E5C2E2E5C2E2E5CC6
:10D6C0002E2E5C536F757263655C6170705F636F63
:10D6D0006D6D6F6E5C6170705F7363686564756CAF
:10D6E00065722E6300000000F0B5002201230326BE
:10D6F00036041F469740394212D0C5683D4203D1D7
:10D70000012464043D4301E03446BD43C560914DAE
:10D7100097007D192F68B7432F602F6827432F602C
:10D72000521C202AE5D3F0BDF8B58B4805698B491A
:10D730000020C863074632E014213A464A43416854
:10D74000806854180121B940014226D0E068C643E0
:10D7500020686E40064031462046FFF7C5FF7E48F0
:10D76000006968400CD00543E0682168C043684008
:10D770000840014600902046FFF7B6FF0098064398
:10D780003046A168A84301402A46606832401040F4
:10D7900002460A4301D0226990477F1CFFB27048BD
:10D7A00041788F42C8D3F8BDF0B56D4A0021536867
:10D7B000142250430124674D03273F041E5822467C
:10D7C0008A40164206D08A0052191668BE43166077
:10D7D00016681660491C2029F0D3F0BD10B5002949
:10D7E00003D08A070024002A01D0072010BD5C4A1C
:10D7F0000B465160107014215470414318469460D8
:10D8000001F0E9FC00205749C04388605648402198
:10D810000160564A1068FF231B0498430B04184309
:10D82000106053480160002010BDF8B54C4F84468D
:10D830007D68002D07D0002B07D078783C78A04277
:10D8400005D30420F8BD0820F8BD0720F8BD0E461A
:10D850001424164344432E5164192361A26061606D
:10D8600061460870411C7970FFF79EFF0020F8BDEB
:10D87000F0B53B4A5168002904D05378984203D34D
:10D880000720F0BD0820F0BD344B0025DD63324B8E
:10D890001C699768002F02D1324EDB0573600126A8
:10D8A00086403E439660142250434218D5600022C1
:10D8B00001230D5893401D4215D01C4202D0032570
:10D8C0002D0405E001256D044618F7681F43F76035
:10D8D000204B9600F3181E6803273F04BE431E60CA
:10D8E0001E682E431E60521C202AE1D30020F0BD8A
:10D8F00070B51B4C05466068002804D060788542EE
:10D9000003D3072070BD082070BD2846FFF74CFFE9
:10D910000121A068A9408843A06003D101201149DA
:10D92000C0078860002070BD0D4B5A68002A04D0E3
:10D930005B78984203D30720704708207047142370
:10D9400058438018044A12690068024000200A60A7
:10D950007047000000070050000500504061004083
:10D960006C2000200063004080E200E004E400E05E
:10D9700000E100E010B50446002A02D01088002221
:10D9800010E00A48FBE7030A00020343A05C58408A
:10D9900003061B0F43401803584083B21806C00CFF
:10D9A0005840521C8A42EED310BD0000FFFF000019
:10D9B00010B508461146FEF78BFC10BDF8B53D4C7E
:10D9C0002078002837D02069002807D00026E0689A
:10D9D000002805D00025002E04D013E00126F6E72C
:10D9E0000125F8E7684651DF052806D0002806D053
:10D9F00031A26921FEF766FC04E0012602E02169FC
:10DA000000988847002D12D1608869460880A06878
:10DA100061DF052806D0002806D027A28021FEF766
:10DA200051FC04E0012502E0E168A0688847002E6F
:10DA3000D8D0002DCFD0F8BD70B5002901D08C070B
:10DA400001D0072070BD1B4C0125A16062802849D0
:10DA5000636010DF0028F5D12570162026DF70BD29
:10DA600011DF002801D0012100E00021114A1170CE
:10DA70007047002803D00F49C860002070470E206F
:10DA80007047002803D00B490861002070470E2022
:10DA9000704710B507484068002808D08047002824
:10DAA00004D0FF2104A23331FEF70CFC10BDFFF7B8
:10DAB00085FF10BD782000202E2E5C2E2E5C2E2E91
:10DAC0005C2E2E5C2E2E5C536F757263655C7364E6
:10DAD0005F636F6D6D6F6E5C736F6674646576699E
:10DAE00063655F68616E646C65722E6300000000A0
:10DAF000B1D9010018225043FA4A0021801801715F
:10DB000081604161012281610261C1607047FFB59E
:10DB100081B0F54C049B039A054626691A430320FD
:10DB20000092002E03D1002A0ED001222261276923
:10DB3000039A0126360792003B0001F042FC0727BA
:10DB400007162940526127000222EFE77069326907
:10DB500092B25043326933691204920C9BB259431A
:10DB600021DF002812D102210FE0084620DF002823
:10DB70000CD10399002901D0032106E00499002962
:10DB800016D12978042946D017E0216105B0F0BDEF
:10DB90007069326992B25043326993B24B43014685
:10DBA0001846039A21DF0028F0D10499002901D0FA
:10DBB0000421EAE72978042920D00521E5E77369E3
:10DBC0003069366980B2434368681B189B18B6B247
:10DBD0004E43301880181946049A21DF0028E9D0F6
:10DBE000D4E7306980B24843696880188A08696957
:10DBF00021DF0028CAD1009900290CD00621C4E7F2
:10DC00007069316989B24843316989B201F0F6FA25
:10DC100020DF0028BAD10721B7E7F8B5B1491823AA
:10DC20000A780F205A435418AF4922796669241D97
:10DC3000CF68022A1BD001252D07042A2AD0052AE5
:10DC40005BD1286981B2304601F0D8FA0146A36859
:10DC500028699A1980B24843101A82086068181817
:10DC6000861928694B1C80B25843801B34E0B802E7
:10DC700062686169121A0918A3683018181801231C
:10DC80009B029A4202D2920821DF31E0FF22013248
:10DC900021DF2DE0E268934914205043F43140180D
:10DCA000001D0BC8B04203D160685943814218D0AF
:10DCB000022A16D0286981B2304601F09FFA014647
:10DCC000286980B24843301A820828694B1C80B208
:10DCD000584363689B19C01A83082046FFF717FF53
:10DCE00006E0286981B2304601F088FAC01920DFC9
:10DCF000002802D17B4901228A70F8BDF8B5794C21
:10DD0000069E65780A2D1DD027787D19EDB20A2D63
:10DD100001D30A3DEDB218277D432D192871AA6160
:10DD200003C9EE60AB6069612861A1780020002919
:10DD300004D1FFF772FF112800D100206178491C3F
:10DD40006170F8BD0420F8BD38B502466548182357
:10DD500001785943081803690179022B0AD0142469
:10DD60006343604CF434E458836800938369103053
:10DD7000A04738BD5C4B14331C68F5E7F8B5594B28
:10DD80009978012914D1002557499D700A69082AFC
:10DD900005D002280FD003280AD10D2006E0022862
:10DDA00007D00D7000F08AFA002801D0FFF7CCFFF1
:10DDB000F8BD0D61F6E74B48182403784A496343E0
:10DDC000CC681818641CCC600379001D022B05D1A7
:10DDD0004668A102B14201D3012700E00027052BCC
:10DDE00001D1072A03D00021042B02D003E0012136
:10DDF000FAE7072A03D00026042B02D007E0012609
:10DE0000FAE74068A302834201D3002A1AD0002017
:10DE1000314301433943C5D0334E28463561FFF7BE
:10DE200093FF304C2078FFF765FEF5606078401E68
:10DE300060702078401CC0B220700A28B2D30A3823
:10DE40002070AFE70120E3E770B50025264C254898
:10DE5000E56025610570457085702E463046FFF7F8
:10DE600049FE761C0A2EF9D301221207656051691A
:10DE700028461269491E92B25143E560A1601949D2
:10DE8000F4310D608D600D61CD60174914310D6066
:10DE9000888001212170206170BDF0B5124A13788D
:10DEA000002B23D0002823D0002921D00368002B89
:10DEB0001ED00124240743682569ADB2AB420FD8B8
:10DEC000102B0DD38568002D0AD092685D436669DA
:10DED000AD182769BFB27E43B54201D89B0709D070
:10DEE0000720F0BD382500208C2000200820F8E70E
:10DEF0000E20F6E7FA4D6B68012B1BD00B604A60D1
:10DF0000194614256943F74D4E19726007686F5022
:10DF10004168B1608168F1604168806800254143D3
:10DF20006D1C2069ADB280B2884205D2206980B2F2
:10DF3000091A02E00420D4E70021206980B2821887
:10DF4000206980B28842EBD9E5485B1C826035616C
:10DF500043600020C5E730B5E14B1B78002B07D0AC
:10DF6000002807D0002A05D00468002C12D103E055
:10DF7000082030BD0E2030BDDA4B1D68002D09D0C1
:10DF80004568986841436918DD6845435868281812
:10DF9000884201D8072030BD14600020516030BD98
:10DFA000F8B50446CE481E46007815460F460028B0
:10DFB00007D0002F07D0002C05D02068002817D1EB
:10DFC00003E00820F8BD0E20F8BDC648016800290E
:10DFD0000ED0C268816840684A4310186268904257
:10DFE00006D9002D04D0A94202D3A819884201D92C
:10DFF0000720F8BD384600F05BF9002811D0304604
:10E0000000F056F900280CD0606800F051F90028A3
:10E0100007D02B463A46214602200096FFF76EFEB7
:10E02000F8BD1020F8BDF8B50446AD481E4600788E
:10E0300015460F46002807D0002F07D0002C05D02A
:10E040002068002817D103E00820F8BD0E20F8BD95
:10E05000A448016800290ED0C268816840684A431C
:10E0600010186268904206D9002D04D0A94202D34C
:10E07000A819884201D90720F8BD384600F018F9E0
:10E08000002811D0304600F013F900280CD0606849
:10E0900000F00EF9002807D02B463A46214605200D
:10E0A0000096FFF72BFEF8BD1020F8BDFFB58C4899
:10E0B00081B000781F4616460D46002808D0002D76
:10E0C00008D00198002805D02868002817D103E05F
:10E0D00008205BE50E2059E5824C206800280ED010
:10E0E000E168A0686268414389186A68914206D96C
:10E0F000002E04D0B04202D3F119814201D9072089
:10E1000044E5019800F0D4F800281BD0384600F010
:10E11000CFF8002816D0686800F0CAF8002811D09F
:10E1200068683246C119019800F0F6FF0096286829
:10E13000142148432458002203212846019BA0476C
:10E14000002023E5102021E5F8B5054664480F4678
:10E150000078002805D0002D05D02868002821D19E
:10E1600003E00820F8BD0E20F8BD5E4C00262068B4
:10E17000002817D0A168E0684843616841186868C2
:10E1800081420FD900F094F800280DD0296814229C
:10E190005143091968684A688968801A01F02EF8A5
:10E1A000002903D00720F8BD1020F8BD3B4600220F
:10E1B000294604200096FFF7A1FDF8BD48490978DB
:10E1C000002907D0002807D04649F4394978016072
:10E1D00000207047082070470E207047404A127890
:10E1E000002A0DD000280DD000290BD00268002A8B
:10E1F00008D03B4A14321368002B05D00420704726
:10E20000082070470E20704702230B6000681060E2
:10E2100000207047F8B5044631481E46007817467E
:10E220000D46002807D0002D07D0002C05D020680F
:10E2300002281BD103E00820F8BD0E20F8BD2848B5
:10E2400014300068002811D0084600F031F800288A
:10E250000ED0304600F02CF8002809D03B462A4664
:10E26000214602200096FFF749FDF8BD0720F8BDC2
:10E270001020F8BD08B51A4A1278002A05D00028E7
:10E2800005D00268022A11D103E0082008BD0E2043
:10E2900008BD134A14321268002A07D00B46002228
:10E2A000014604200092FFF729FD08BD072008BDA4
:10E2B000800701D00020704701207047094810B541
:10E2C000F43840780024002807D0FFF7A6FC0400AB
:10E2D00003D0112C01D0FFF737FD204610BD000000
:10E2E0008C2000202C260020564800210170574821
:10E2F000554A02608160C16001610822416142604B
:10E3000081610846704700207047002805D04D49BC
:10E310000A78002A03D0042070470E20704701229B
:10E320000A704849491C0160002070474549002097
:10E330000870704710B500291DD000220A60434ABA
:10E340005368002B1BD0202817D85B1E5360D06861
:10E350002423401CD060106914684343E3180B6009
:10E36000012383409169401C19434007400F91618C
:10E370001061002010BD0E2010BD0C2010BD042027
:10E3800010BDF0B5314A0646916800292AD0576978
:10E390001020791A4907490F14680B4624254D436C
:10E3A0006519B54206D1012495698C40654000206D
:10E3B000956104E0491C4907490F8F42EED1491C81
:10E3C0004E07760F956901210C469C4025420AD1E3
:10E3D0009368002B07D05B1E936053685B1C5360EF
:10E3E0003346F1E70420F0BD184A2423117C12685B
:10E3F000491E4907490F59432031505000207047AA
:10E4000070B500281AD0002918D0104AD368002B04
:10E4100016D05B1ED360936824265B1C93605369FF
:10E4200015681C467343EE1820330660E858641CD8
:10E4300008606007400F5061002070BD0E2070BD65
:10E44000042070BDA8200020402600206027002066
:10E4500010B500280BD0FE48FE49808888420FD0B6
:10E46000132176DF00280BD0FBA2702106E00846BE
:10E47000FFF787FF002803D0F7A27621FDF722FFE0
:10E4800010BD08280CD004DC002807D006280FD1C6
:10E4900008E00B280AD00C280AD105E001207047BB
:10E4A000022070470320704704207047042901D0E0
:10E4B000062070470520704710B5E54A00280AD0AD
:10E4C0009088E449884215D0132176DF002811D0C6
:10E4D000E1A2B4210CE001215069FFF7D2FF02460E
:10E4E0000121E348FEF766FA002803D0DAA2C12131
:10E4F000FDF7E8FE10BDF0B5054608790E4685B07B
:10E5000081070AD0032211462846FEF753FA002855
:10E5100021D0FF21D0A24B3146E0CD4900901031EF
:10E52000FFF708FF010013D1C94CB168009A2069B8
:10E5300000F0F2FD0098FFF757FF002801D00146D8
:10E5400006E0C34869461030FFF75AFF010004D0C7
:10E55000284600F0C6F905B0F0BD0098800802908A
:10E56000032001902069039001A8FEF76DF80700D1
:10E570000CD0092F1BD02069FFF703FF002803D020
:10E580000146284600F0ADF93946E1E73079E188E7
:10E5900001224018E08003212846FEF70BFA0028EC
:10E5A000D9D0FF21ACA27B31FDF78CFED3E73079C7
:10E5B000E188401881B2E18060780028CBD0608982
:10E5C000401E0004000C6081C5D12846FEF731FBD7
:10E5D000002804D0FF21A0A28C31FDF773FE208912
:10E5E0006081B8E710B5FF219BA2C731FDF76AFE35
:10E5F00010BD10B5964C9749A088884208D01321C9
:10E6000076DF002814D094A29A49FDF75BFE0FE054
:10E61000A07800280CD074DF002803D096A29C4973
:10E62000FDF750FE01209B490004C8600020A07047
:10E6300000F08DFA002804D08E4987A20931FDF739
:10E6400041FE002010BD70B50D68044601228048CF
:10E650002B0000F0B6FE0A3032340616243B403759
:10E660004423FEF740F80421FFF70BFF0246042184
:10E670002046FEF79FF9002810D0FF2176A2F9313D
:10E6800036E0FFF7B6FF002804D0FF2172A2FF3169
:10E69000FDF718FEFEF748F8002809D170BDFFF716
:10E6A000A8FF002804D07A496BA24739FDF70AFE7B
:10E6B000FEF74DF870BDC26070BD022100E003217D
:10E6C000C16070BD204600F01FF970BD427089889E
:10E6D0000181418170BD00214170018170BDC188FF
:10E6E0002046FEF76FFA0028F8D08B215AA2890045
:10E6F000FDF7E8FD70BD10B5554CA07800280ED18F
:10E700005B48143873DF002804D0614952A21239E3
:10E71000FDF7D8FD01205F4A01049160A07010BD93
:10E7200070B54B4C0588A388132D2CD00ADC5A4AAF
:10E730005849102D18D0112D15D1CA602078002805
:10E740001BD01CE0522D29D0552D0CD180790028EA
:10E7500009D11321184676DF002804D051213EA2AA
:10E76000C900FDF7AFFD70BD8A6001221204CA60C6
:10E770008088A0800020A07070BDFFF7BCFF002043
:10E78000C043A08070BD324A1846183200217FDF96
:10E790000028F7D0052130A2C901E2E70022114686
:10E7A0001846A9DF0028EDD039492BA23D31D8E722
:10E7B00010B5044600F0FCF921462D48FEF7C8F9D3
:10E7C0002046FFF7ADFF10BD2A4910B522A25039EF
:10E7D000FDF778FD10BD30B51D4887B00024C4603A
:10E7E0002E4803250560001F056005602C48FFF7D3
:10E7F00040F9002873D12B48FDF7FFFE2A48FDF7AA
:10E80000FFFEFFF771FD002869D100F0A7F8274847
:10E8100000902748019069461548FEF75FF90028E7
:10E8200004D0144914A23D39FDF74CFD00F0BAF8AC
:10E830001C21684600F0CFFC1E4801900120800397
:10E840000290009468460573C48104741A4835E048
:10E85000B0200020FFFF00002E2E5C6466755F7400
:10E8600072616E73706F72745F626C652E6300000C
:10E8700090270020520300002E2E5C6466755F74A2
:10E8800072616E73706F72745F626C652E630000EC
:10E8900051020000000500500080000040070050B9
:10E8A000B1E7010051E40100B9E4010047E60100CD
:10E8B000C9E70100CD0C0000E5E5010006900594D4
:10E8C000684600F020F9002804D0FF21714ADE31AB
:10E8D000FDF7F8FC00F09BF8FFF70DFF002007B0F4
:10E8E00030BD10B50A46044603211046FFF7C9FDA6
:10E8F000024603212046FEF75DF8002803D0654A52
:10E90000D821FDF7DFFC10BD70B5634DEA68012A20
:10E9100006D0022A1FD0032A01D1FFF7ECFD70BDFB
:10E920000A79042A0AD003220121FEF743F80028BD
:10E93000F5D0584AEC21FDF7C5FC70BD8C68204627
:10E9400000F04BFCE1780002000A09060843FDF7DD
:10E950005AFE686170BD00F06CF870BD0EB51120F4
:10E960006946087207224DA102A87CDF002804D066
:10E97000B121484A8900FDF7A5FC0020009009223A
:10E98000694601900A800C224A808880FF209130DD
:10E99000C88068467ADF002803D03E4A4149FDF727
:10E9A00091FC0EBD10B592B00621684601713E483B
:10E9B0000179684681703D4901803C2102A800F040
:10E9C0000AFC02200290002468464473012101825F
:10E9D00001A80590684681830890214602A800F0AE
:10E9E0007DFA002804D0BB212A4A8900FDF76AFC81
:10E9F0002D481421143800F0EEFB2B481438047015
:10EA00004460047228210182448212B010BD224960
:10EA10001E2018310880887801221043E12210401E
:10EA2000DF220C30104088700720C8701020087159
:10EA30007047FEB50446012000908868029008796E
:10EA4000002283070FD08007800F0422121A0020B3
:10EA5000034606E00E79029D3618B600401CAB5105
:10EA6000C0B29042F6D308798018800801906846B9
:10EA7000FDF718FE0221FFF704FD024602212046A1
:10EA8000FDF798FF002804D0FF21024A3631FDF738
:10EA900019FCFEBD78E80100B020002044667554E2
:10EAA00061726700CE020000902700203015000040
:10EAB00038B57A497A4A488890420FD04A78794CDA
:10EAC000521CD2B24A70237B934208D3083175DFBF
:10EAD000002803D0A169002900D0884738BD00254F
:10EAE0004D70217C002907D03B2176DF002803D020
:10EAF000A169002900D0884761690029EED06846E5
:10EB00000095884738BD70B5054601461C2265480A
:10EB1000FDF73EFB614C002626702968002907D0CE
:10EB20000822A01800F0F8FA204608307ADF02E048
:10EB30005A4808307BDF002808D1401E60805748C3
:10EB40006670594A0021001DFEF7CBFA70BD10B562
:10EB500052484068FEF774FB10BDF8B54F481030BE
:10EB600000F08EF800264D4D4E4C002806D061690D
:10EB7000002919D001200090684614E02878002868
:10EB800004D0616900290FD00096F5E76878002865
:10EB90000CD0A16800226868FEF7EAFA002803D0CA
:10EBA000A169002900D088472E70F8BD6168F1E79F
:10EBB000F8B53C4C02880027384DE689102A18D059
:10EBC00029464968112A21D0122A2DD0502A0FD166
:10EBD000C288801DB2420BD1028B022A08D1C27EAC
:10EBE000837E10021843C007C00F13D0FFF7B5FF94
:10EBF000F8BD818869800146284808220E3110300E
:10EC000000F08AFA6F70002EF0D0F8BD0020C043EB
:10EC100068806F700846FEF713FB0028F5D0A169E5
:10EC20000029F2D08847F8BD811D1C480822103009
:10EC300000F072FADAE7F8B5014618480822083001
:10EC400000F06AFA154808307ADF04000DD1134845
:10EC5000103000F015F80125002808D0114841694E
:10EC6000002902D06846009588472046F8BD0B4E23
:10EC7000357031460831708875DF04467570F4E7E9
:10EC80004188064808300288914204D34088814276
:10EC900001D801207047002070470000D0200020DC
:10ECA000FFFF0000B8270020B1EA0100FFB583B0E4
:10ECB000074600200C9C8646267805463AE0786890
:10ECC000A90041180A88684682804988C1800022CC
:10ECD000694601A865DF002810D1684601780598CB
:10ECE000814226D17046002801D0002200E0022295
:10ECF0002078891841181F2902D90C2007B0F0BDCF
:10ED00007146002908D1401CC0B2411C069B049AE0
:10ED100021701A5401208646217806980A186946FF
:10ED200001A865DF0028E9D16946207809784018F4
:10ED300020706D1C3888A842C1DC7046002804D0C1
:10ED400020780699801B401E88550020D6E7F8B52C
:10ED50001546069C1E46074602220094FFF7A6FFB2
:10ED6000002806D133461022294638460094FFF782
:10ED70009DFFF8BDF7B582B0002605461670006805
:10ED80001446002805D02846039900F0DFF8060055
:10ED90002DD1687900281BD02078039F001D1F28E3
:10EDA00024D8684679DF002821D121780322481C25
:10EDB00020707A5421781922481C20707A542078C7
:10EDC000C1196846008800F0BCF82178401820700E
:10EDD0002989002923D001208446EA680398002A63
:10EDE00007D0227853189B1C1F2B04D90C2005B088
:10EDF000F0BD0720FBE71346521C2270491CC1548A
:10EE000022786746511C2170875423782A89181864
:10EE1000E96800F081F92078297A40182070286983
:10EE2000002815D00021415622788C46D01C039929
:10EE30001F28DBD8501C022320708B5422780A2311
:10EE4000501C20708B5420786246431C23700A5457
:10EE5000A88A002809D028460094062202211430EE
:10EE6000039BFFF774FF0600C1D1A88B002809D0CF
:10EE700028460094072203211C30039BFFF767FFFD
:10EE80000600B4D1A88C002809D028460094152289
:10EE900014212430039BFFF75AFF0600A7D1E86A2C
:10EEA000002805D02246039900F085F806009ED17F
:10EEB000286B002805D02246039900F0BBF8060015
:10EEC00095D13820405D002806D022462846039977
:10EED00000F0E2F806008AD1304688E770B50D46AA
:10EEE00092B000216A46117007241171002812D0D7
:10EEF0000189002905D0C168002902D00978490795
:10EF000002D4204612B070BD02A9FFF733FF0028DB
:10EF1000F8D102AE00E00026002D0BD02889002891
:10EF2000EFD101AA0AA92846FFF724FF0028E9D15A
:10EF30000AAA00E00022684603790178304672DFB1
:10EF4000E0E70870000A487002207047F8B51478AE
:10EF50000746A01C15460E461F2803D83879801C8A
:10EF60001F2801D90C20F8BD1D20001B80B2694666
:10EF7000864608803019801C7DDF0028F3D1386870
:10EF8000022805D168460088704501D8092107E0AC
:10EF900038790821002801D0704501D968460088D9
:10EFA000421C3255641CE2B2B1542978801C081806
:10EFB00028700020F8BDF8B50D4611780646881D6A
:10EFC00014461F2801D90C20F8BD33880720062BD2
:10EFD000FAD31927FF01BB4202D94E4A9342F3D11B
:10EFE0007288062AF0D3BA4202D94A4FBA42EBD10C
:10EFF000484FBB4203D0BA4201D09342E4D8481CE8
:10F00000052220706A5420781222411C21702A5453
:10F01000207841193088FFF794FF21784018C0B25A
:10F02000207041197088FFF78CFF217840182070FC
:10F030000020F8BD70B5054600790E46801C1446C8
:10F04000C0B21178821C8A181F2A01D90C2070BD09
:10F050000A46491C2170401CB0542078FF22411CF4
:10F0600021703254207881192888FFF76AFF2178AF
:10F070004018C0B22070AA88002A09D0A9680029C7
:10F0800008D0801900F048F82078297940182070BD
:10F09000002070BD072070BDF7B582B002981446FD
:10F0A000406B0F46002832D0029800252030009097
:10F0B00028E00298416B0C2068430E1821783079C3
:10F0C0004A1C2270C01C785420781622411C2170E2
:10F0D0003A542078C1193088FFF733FF217840185F
:10F0E000C0B22070B288002A09D0B16800290ED0C1
:10F0F000C01900F011F820783179401820706D1C8B
:10F100000098EDB2007EA842D3D800206FE6072019
:10F110006DE60000FFFF0000F8B5042A2CD383073A
:10F1200012D00B78491C0370401C521E83070BD071
:10F130000B78491C0370401C521E830704D00B78C7
:10F14000491C0370401C521E8B079B0F05D0C91A27
:10F15000DF002023DE1B08C90AE0FDF719F8F8BD1F
:10F160001D4608C9FD401C46B4402C4310C0121F68
:10F17000042AF5D2F308C91A521EF0D40B78491CA0
:10F180000370401C521EEAD40B78491C0370401CCB
:10F19000012AE4D409780170F8BD01E004C0091F18
:10F1A0000429FBD28B0701D50280801CC90700D03F
:10F1B0000270704700290BD0C30702D00270401CB8
:10F1C000491E022904D3830702D50280801C891EB0
:10F1D000E3E70022EEE70022DFE70378C278194672
:10F1E000437812061B0219438378C0781B04194325
:10F1F00011430902090A0006084370470022030967
:10F200008B422CD3030A8B4211D300239C464EE041
:10F2100003460B433CD4002243088B4231D30309FD
:10F220008B421CD3030A8B4201D394463FE0C309AF
:10F230008B4201D3CB01C01A524183098B4201D3C7
:10F240008B01C01A524143098B4201D34B01C01AB2
:10F25000524103098B4201D30B01C01A5241C3082A
:10F260008B4201D3CB00C01A524183088B4201D399
:10F270008B00C01A524143088B4201D34B00C01A85
:10F280005241411A00D201465241104670475DE09A
:10F29000CA0F00D04942031000D34042534000221D
:10F2A0009C4603098B422DD3030A8B4212D3FC22C6
:10F2B000890112BA030A8B420CD3890192118B4245
:10F2C00008D3890192118B4204D389013AD092115B
:10F2D00000E08909C3098B4201D3CB01C01A524116
:10F2E00083098B4201D38B01C01A524143098B42DF
:10F2F00001D34B01C01A524103098B4201D30B01C8
:10F30000C01A5241C3088B4201D3CB00C01A5241EC
:10F3100083088B4201D38B00C01A5241D9D24308D3
:10F320008B4201D34B00C01A5241411A00D2014610
:10F33000634652415B10104601D34042002B00D57A
:10F340004942704763465B1000D3404201B500203C
:10F35000C046C04602BD704770477047754600F012
:10F3600025F8AE46050069465346C008C0008546EC
:10F3700018B020B5FCF790FF60BC00274908B646DE
:10F380000026C0C5C0C5C0C5C0C5C0C5C0C5C0C5B4
:10F39000C0C5403D49008D46704710B50446C04683
:10F3A000C0462046FCF7D7FE10BD0000004870475D
:10F3B000D427002001491820ABBEFEE7260002003A
:10F3C000704730B47446641E2578641CAB4200D28A
:10F3D0001D46635D5B00E31830BC18470200000067
:10F3E00000000000000000000000000023D1BCEA83
:10F3F0005F782315DEEF1212000000001CF40100FC
:10F4000000200020E800000004C1010004F5010014
:10F41000E82000205013000020C101000024F40067
:10F4200000000000000000000000000000000000DC
:10F4300000000000000000000000000000000000CC
:10F4400000000000000000000000000000000000BC
:10F4500000000000000000000000000000000000AC
:10F46000000000000000000000000000000000009C
:10F47000000000000000000000000000000000008C
:10F48000000000000000000000000000000000007C
:10F49000000000000000000000000000000000006C
:10F4A000000000000000000000000000000000005C
:10F4B000000000000000000000000000000000004C
:10F4C000000000000000000000000000000000003C
:10F4D000FFFF00000000000000000000000000002E
:10F4E000000000000000000000000000000000001C
:10F4F000000000000000000000000000000000000C
:04F500000000000007
:020000041000EA
:0410140000C0010017
:040000050001C0C175
:00000001FF
